:020000040800F2
:10000000D84F00206102000847220008D9200008CC
:1000100045220008450D00081924000800000000D2
:10002000000000000000000000000000A101000826
:10003000010E000800000000FD010008B9220008C0
:100040007B0200087B0200087B0200087B0200089C
:100050007B0200087B0200087B0200087B0200088C
:100060007B0200087B0200087B0200087B0200087C
:100070007B0200087B0200087B0200087B0200086C
:100080007B0200087B0200087B0200087B0200085C
:10009000490D0008550D00087B0200087B0200088E
:1000A0007B0200087B0200087B0200087B0200083C
:1000B0007B0200087B0200087B0200087B0200082C
:1000C0007B0200087B0200087B0200087B0200081C
:1000D0007B0200087B0200087B0200087B0200080C
:1000E0007B0200087B0200087B0200087B020008FC
:1000F0007B0200087B0200087B0200087B020008EC
:100100007B0200087B0200087B0200087B020008DB
:100110007B0200087B0200087B0200087B020008CB
:100120007B0200087B0200087B0200087B020008BB
:100130007B0200087B0200087B0200087B020008AB
:10014000610D00086D0D00087B0200087B020008AD
:100150007B0200087B0200087B0200087B0200088B
:100160007B0200087B0200087B0200087B0200087B
:100170007B0200087B0200087B02000800000000F0
:100180007B0200087B020008DFF810D000F050FB73
:10019000004800474D280008AFF30080D84F0020EA
:1001A0002C4B19680868B0E8F04F80F30988BFF35A
:1001B0006F8F4FF0000080F311887047000000003F
:1001C00008480068006880F308884FF0000080F35A
:1001D000148862B661B6BFF34F8FBFF36F8F00DF35
:1001E00000BF00BF08ED00E0DFF80C00016841F43B
:1001F00070010160704700BF88ED00E0EFF30980F7
:10020000BFF36F8F134B1A681EF0100F08BF20ED5D
:10021000108A20E9F04F106009B44FF0500080F3CD
:100220001188BFF34F8FBFF36F8F03F067FC4FF060
:10023000000080F3118809BC19680868B0E8F04F25
:100240001EF0100F08BFB0EC108A80F30988BFF3CE
:100250006F8F704718000020EFF305807047000093
:100260000648804706480047FEE7FEE7FEE7FEE750
:10027000FEE7FEE7FEE7FEE7FEE7FEE76523000890
:10028000890100082DE9F05F0546002092469B4653
:1002900088460646814640241BE02846414647469C
:1002A000224600F0BEF953465A46C01A914110D377
:1002B00011461846224600F0A5F92D1A67EB0108F1
:1002C0004F4622460120002100F09CF917EB00095F
:1002D0004E41201EA4F10104DFDC484631462A4687
:1002E0004346BDE8F09F40EA01039B0703D009E0C5
:1002F00008C9121F08C0042AFAD203E011F8013B12
:1003000000F8013B521EF9D27047D2B201E000F86A
:10031000012B491EFBD270470022F6E710B51346A9
:100320000A4604461946FFF7F0FF204610BD2DE9A6
:10033000FE4F804681EA0300C00F0C46009021F07A
:10034000004123F00045B8EB0200A94105D2404628
:10035000214690461C460B46024623F000401043BF
:1003600047D0270DC7F30A00C3F30A510290401A81
:10037000019040286BDAC3F3130040F4801B00980F
:10038000924620B10023D2EB030A63EB0B0B0198DA
:100390005946C0F14002504600F034F906460D4679
:1003A00050465946019A00F04CF910EB08006141A3
:1003B000002487EA115284EAE7731A4340D0009A76
:1003C00062B3019A012A4FEA075215DC001B61EB68
:1003D00002014FF0004202EA0752CDE90042001C40
:1003E00041F5801132462B4600F083F903B0BDE899
:1003F000F08F40462146F9E7001B61EB0201001C2B
:1004000041F5801300185B412018A2F5001747EB57
:10041000030140EAD570B6196D4111E06D084FEA4D
:10042000360645EAC0754FEA0752001B61EB020130
:10043000001C41F5801149084FEA30000019514174
:1004400032462B4603B0BDE8F04F00F043B90098A8
:10045000012240000023D0EB020263EBE07300981E
:1004600021464FEAE074B8EB000061EB0401E9E7D4
:1004700083F000435BE781F0004158E72DE9F04D40
:1004800081EA030404F0004B21F0004514464FF0CC
:10049000000A23F0004150EA050220D054EA01028C
:1004A0001DD0C5F30A570246C5F31303C1F3130069
:1004B000C1F30A5640F4801543F48013A7EB0608F5
:1004C000101BD64608F2FD3873EB050002D308F185
:1004D000010801E092185B41B8F1000F03DA002037
:1004E0000146BDE8F08D00204FF480110646844699
:1004F0000EE0171B73EB050705D3121B63EB050317
:1005000006434CEA010C49084FEA300092185B415F
:1005100050EA0107EDD152EA030012D082EA04004A
:1005200083EA0501084305D0101BAB4106D2012226
:10053000002306E000224FF0004302E06FF00102CA
:1005400053101AEB06004CEB085110EB0A0041EB7C
:100550000B01BDE8F04D00F0BDB80EB540F23341DF
:1005600002910021CDE900110A460B4600F0C1F8C6
:1005700003B000BDC1F30A5210B5C1F3130140F23C
:10058000FF3341F480119A4201DA002010BD40F29D
:1005900033439A42A2F2334203DC524200F041F864
:1005A00010BD904010BD00F0004230F000400AD075
:1005B000C10D01F56071C0F3160042EA0151C20895
:1005C00040071143704700200146704701F0004387
:1005D00030B421F0004150EA010206D00A0DA2F524
:1005E0006072C1F31301002A02DC30BC00207047A6
:1005F000440F44EAC104C100E01830BC00EBC25013
:1006000000F031B8202A04DB203A00FA02F1002081
:1006100070479140C2F1200320FA03F31943904040
:100620007047202A04DB203A21FA02F000217047AB
:1006300021FA02F3D040C2F120029140084319464A
:100640007047202A06DBCB17203A41FA02F043EA32
:10065000E07306E041FA02F3D040C2F1200291407B
:100660000843194670470029A8BF7047401C49003D
:1006700008BF20F00100704710B4B0FA80FC00FA07
:100680000CF050EA010404BF10BC704749B1CCF132
:10069000200421FA04F411FA0CF118BF01212143BE
:1006A0000843A3EB0C01CB1D4FEA00614FEA102079
:1006B00042BF002010BC704700EBC350104400291B
:1006C000A4BF10BC7047401C490008BF20F00100C7
:1006D00010BC704710B5141E73F1000408DA401CFA
:1006E00041F1000192185B411A4301D120F0010051
:1006F00010BD2DE9F04D92469B4611B1B1FA81F241
:1007000002E0B0FA80F220329046FFF77BFF044609
:100710000F4640EA0A0041EA0B0153465A46084395
:1007200013D0114653EA010019D0C8F140025046D7
:10073000FFF777FF05460E46504659464246FFF7FB
:1007400061FF084305D0012004E020463946BDE89A
:10075000F08D0020054346EAE0762C4337430A98A3
:100760006305E40AA0EB08000022FD0A44EA4754AE
:100770000A3002D500200146E9E701051019694158
:10078000DDE9084500196941BDE8F04DA2E72DE912
:10079000F04D00231A461B1A8A4103DB0020014654
:1007A000BDE8F08DC1F30A52C1F3130141F4801585
:1007B0004FF0000BD10702D100186D41521E0027E7
:1007C000044640F2FF11384601EB620A3E4680467D
:1007D000024600204FF48011FFF723FFC219714138
:1007E000BB1846EB0100B4EB030C75EB000C04D313
:1007F000E41A65EB000517460E46241908F10100BE
:100800006D4180463428E3DDF91946EB0600091BEB
:10081000A84103D24FF0FF32134601E000221346F5
:100820001BEB070046EB0A51BDE8F04DFFF752BF46
:10083000064C074D06E0E06840F0010394E807002D
:1008400098471034AC42F6D3FFF7A2FC8C4900085D
:10085000AC4900082DE9F04716008846074600D14C
:100860000A261F4C6421A06802F026F918B16FF027
:100870000400BDE8F0874FF0FF3960680BE00178B5
:10088000B94207D14268424504D1A06802F071F92B
:100890004846EEE700690028F1D1142000F050FA34
:1008A000050012D000221C21304602F0A5F8A860F5
:1008B00088B12F70C5F804802E7360682861656068
:1008C000A06802F056F90020D3E7A06802F051F9C1
:1008D0006FF00100CDE7284600F030FAD5E70000C0
:1008E0009800002070470000074A526808E013781B
:1008F000834204D153688B4201D1906870471269DA
:10090000002AF4D10020704798000020C168806858
:10091000022903D0042807D000207047042801D002
:10092000022070470320704701207047022802D23E
:1009300018B1012803D000207047024870470248D0
:1009400070470000E40000200C0100202DE9F04178
:10095000164C07469846207815460E4648B15DB1BC
:100960006421A06802F0A8F848B16FF00400BDE867
:10097000F0816FF00200FAE76FF00100F7E731460F
:100980003846FFF7B1FF0646A06802F0F2F856B10C
:10099000434600222946304601F0FCFF0028E6D0FD
:1009A0004FF0FF30E3E76FF00300E0E7980000202E
:1009B00070B5274C8AB0207818B16FF002000AB0E9
:1009C00070BD68212348FFF7A7FC2348E0600020A2
:1009D00002F09BF8A060B0B301252570282168467D
:1009E000FFF79AFC00200190CDE9060503900490E2
:1009F0000E260590CDE908560090029069461748EA
:100A000000F07CFA154800F03DFE154A0621002052
:100A100000F034F80321114800F0F5F9CDE904564F
:100A20006946104800F06AFA0E4800F02BFE0E4AA4
:100A30000821012000F022F810210A4800F0E3F913
:100A400025700020BBE7FFE74FF0FF30B7E700005D
:100A500098000020184A0020E5080008E400002063
:100A6000D50A00080C010020710B0008024AD26868
:100A7000002A00D010477047980000200E4B1B78CA
:100A800043B152B14FF0FF33022801D20D2907D3F1
:100A9000184670476FF0020070476FF00100704712
:100AA00000EB800303EBC000044B03EB800040F835
:100AB000212000207047000098000020184A0020E4
:100AC000034B1B780BB1FFF7C5BE6FF002007047F8
:100AD000980000202DE9F04391B00024E0B2FFF728
:100AE00025FF06003ED037E00EAB6A4600213046B7
:100AF00000F0B1FA80BB0298E8B1019D6846FFF7AB
:100B000005FF804601462846FFF7B0FF8146E0B268
:100B10004946FFF7E9FE07001ED01C2107A8FFF792
:100B2000FBFBCDE9085904988DF8280003988DF84F
:100B30001C8010B107E0009DE0E70EA90DF129002F
:100B4000049AFFF7D0FB00F05FFF00230D901A46D8
:100B500007A9384601F07CFF0021304600F06AFA10
:100B60000028C1D1641C022CB8DB11B0BDE8F083B1
:100B70002DE9F04391B00024E0B2FFF7D7FE060064
:100B80003ED037E00EAB6A460121304600F063FAF2
:100B900080BB0298E8B1019D6846FFF7B7FE80462A
:100BA00001462846FFF762FF8146E0B24946FFF75B
:100BB0009BFE07001ED01C2107A8FFF7ADFBCDE967
:100BC000085904988DF8280003988DF81C8010B1FE
:100BD00007E0009DE0E70EA90DF12900049AFFF758
:100BE00082FB00F011FF00230D901A4607A938463A
:100BF00001F02EFF0121304600F01CFA0028C1D17F
:100C0000641C022CB8DB11B0BDE8F0832DE9F04381
:100C10000D46264987B0994609780E9F144649B17A
:100C20004FF0FF3802283FD26FF00101B9F1000FF9
:100C300005D008E06FF0020007B0BDE8F083022D98
:100C400001D0032D14D1082F2ED8FFF76FFE060018
:100C50000ED018216846FFF75FFB002055B1042134
:100C6000012D0BD00222022D0CD0032D1CD10DE042
:100C70000846E1E70290009403900AE0CDE90210F3
:100C8000019406E0CDE90202009402E0CDE90212EF
:100C900001948DF81400049706AB4A466946304625
:100CA00000F0C3F80028C7D04046C5E798000020F0
:100CB00008B539B10A7900924B1D0A680021FFF787
:100CC000A5FF08BD6FF0010008BD00002DE9F0414F
:100CD0000C461949097829B1022806D34FF0FF3094
:100CE000BDE8F0816FF00200FAE7FFF71FFE050094
:100CF00006D000F089FE06466FF004071CB10AE03A
:100D00006FF00100ECE7284600F01FFA08B1002060
:100D1000E6E73846E4E7284600F017FA0028F6D15F
:100D2000601C04D000F070FE801BA042F1D20120B4
:100D300001F09FFDEFE700009800002002F0B0BC3A
:100D400002F070BBFEE70000014800F014BA00009A
:100D5000E4000020014800F00EBA0000E40000208A
:100D6000014800F008BA00000C010020014800F022
:100D700002BA00000C01002050B100680549884209
:100D800001D1002070470449884201D101207047F9
:100D90000320704700640040006800401FB548B35E
:100DA0000121009108218DF8041001788DF80510BB
:100DB0004178124A8DF8061081781278891A8DF8D8
:100DC0000710C0788DF8080000208DF809008DF814
:100DD0000A008DF80B008DF80C000121FFF776FF5B
:100DE00069460020FFF764FF002801D04FF0FF3074
:100DF00004B010BD6FF00100FAE70000A800002069
:100E0000704772B6FEE790F82020012A07D0022A28
:100E100005D0416A41F48021416201207047006899
:100E200042690A43426100207047F0B590F82050B3
:100E30000468A468012D05D0022D03D0416A41F455
:100E4000802157E014F0406F01D1E5004FD5C4F385
:100E500001640125A5401D608D684FF4C0739DB1EC
:100E6000CE6835434E6845EAC605066803EB0417AD
:100E7000F5514FF4C275076805EB04150E697E51F4
:100E8000097D012905D009E00E88CD6845EA46555F
:100E9000EBE701684E5946F480764E511179D579C9
:100EA000567941EA056195792D0445EA06252943DD
:100EB0004FF4C676056806EB0416A9511178D5786B
:100EC00041EA0561957852782D0445EA02221143E2
:100ED0004FF4C475026805EB04155151006803EB2B
:100EE0000411425842F0010242500020F0BD416A14
:100EF00041F4001141620120F0BD000010B590F8EE
:100F00002020012A07D0022A05D0416A41F480211D
:100F10004162012010BD3B48D0F8002242F001029E
:100F2000C0F80022D0F8002222F47C52C0F800223F
:100F3000D0F800224B6A42EA0322C0F800220A7D60
:100F400002F01F0301229A40D0F81C329343C0F8EC
:100F50001C32CB69B3B9D0F80C329343C0F80C32D1
:100F60008C894B6864F31F434C6900EBC404C4F8DC
:100F700040320C890B6864F31F434C6900EBC404D6
:100F8000C4F84432CB69012B16D1D0F80C3213438C
:100F9000C0F80C320C884B6864F31F434C6900EBBB
:100FA000C404C4F840320C89CB6864F31F434C6915
:100FB00000EBC404C4F844328B69002BD0F804322F
:100FC0000ED01343C0F804320B69002BD0F8143252
:100FD00008D01343C0F81432096A012904D008E08C
:100FE0009343EFE79343F5E7D0F81C121143C0F8A1
:100FF0001C12D0F8001221F00101C0F800120020EC
:1010000010BD00000064004010B5FFF7B5FE0328D6
:101010000CD000EB800101EBC001054800EB810022
:10102000006B002802D0BDE81040004710BD000052
:10103000184A00200246002092F82030012B01D0EF
:10104000022B05D1106821B1D0F8100000F0030088
:101050007047C068FAE770B590F82040012C05D0C1
:10106000022C03D0416A41F4802128E0046809B3CE
:101070002469A40720D04FF4D874056804EB011448
:101080002D5915F00405956005682D591AD0ED0805
:10109000556005682C5904F00204D4604FF4DA74EA
:1010A000056804EB01142E5906F00F06082E0CD328
:1010B00008250DE0E468DCE7416A41F40011416273
:1010C000012070BD6D0D1560E3E72D5905F00F058A
:1010D000156105682D59C5F30725956105682C59DB
:1010E000240C54614FF4DC72046802EB0112A45822
:1010F0001C700468A458240A5C700468A458240C6A
:101100009C700468A258120EDA704FF4DE72046804
:1011100002EB0112A4581C710468A458240A5C71E3
:101120000468A458240C9C710468A258120EDA7149
:10113000006829B1016941F020010161002070BD02
:10114000C16841F02001C160F8E70246002092F832
:101150002010012901D002290CD111688A6852019E
:1011600000D501208A68120100D5401C8968C90099
:1011700000D5401C70472DE9F05F0546006800244B
:101180004669D0F804908768D0F80CB0D0F810A069
:10119000D0F81880F10748D0F90714D001218160F8
:1011A000B80703D5284600F0AFFA0CE0780702D55F
:1011B0004FF4006407E0380702D54FF4805402E092
:1011C000284600F08BFAF80516D529684FF4807090
:1011D0008860B80503D5284600F0C0FA0CE0780511
:1011E00002D544F4005407E0380502D544F48044A5
:1011F00002E0284600F09CFAF80316D529684FF45F
:1012000080308860B80303D5284600F0D3FA0CE09C
:10121000780302D544F4004407E0380302D544F4CF
:10122000803402E0284600F0AFFA300707D55FEAC5
:10123000CB6004D52968102044F40074C86070079E
:101240004FF0080707D55FEA0B7004D52868C76020
:10125000284600F0A9F9B00706D52868C0688007BD
:1012600002D0284600F0B6F9700607D55FEACA60DA
:1012700004D52968102044F480640861B00607D5BD
:101280005FEA0A7004D528680761284600F0B8F9BB
:10129000F00606D528680069800702D0284600F0CD
:1012A000C5F9B00308D55FEAC96005D529681020E3
:1012B0004860284600F0D0F9F00307D55FEA0970CE
:1012C00004D528684760284600F08AFA300446D5DD
:1012D0005FEA497040D5F00504D55FEAC87001D0D7
:1012E00044F00104B00504D55FEA887001D544F0EC
:1012F0000204700504D55FEA487001D544F0040487
:10130000300529D518F0700F26D008F0700040285D
:1013100015D006DC102809D020280AD0302816D194
:101320000AE050280ED0602811D10EE044F00804E5
:101330000DE044F010040AE044F0200407E044F01B
:10134000400404E044F0800401E044F48074286820
:10135000816921F070018161296804204860002CB6
:1013600005D0686A204368622846FFF74DFEBDE855
:10137000F09F70B5040003D094F8200010B104E091
:10138000012070BD204600F081F82068016841F01E
:101390000101016000F038FB0546052604E000F07D
:1013A00033FB401B0A2811D820684068C007F6D0DC
:1013B0002068016821F00201016000F025FB05466C
:1013C0000BE000F021FB401B0A2806D9606A40F4BC
:1013D0000030606284F82060D2E7206840688007AF
:1013E000EFD4207E0128206801683DD021F08001E3
:1013F0000160607E01282068016838D021F040013A
:101400000160A07E01282068016833D021F020010E
:101410000160E07E0128206801682ED041F01001B3
:101420000160207F01282068016829D021F008018F
:101430000160607F01282068016824D021F0040148
:101440000160D4E902010843D4E9041211430843BE
:101450006168491E08432168C8610020606201205C
:1014600084F82000002070BD41F08001C0E741F009
:101470004001C5E741F02001CAE721F01001CFE7A4
:1014800041F00801D4E741F00401D9E7F0B587B095
:10149000044614216846FEF73FFF3E4B3E48DFF806
:1014A000F0E01968D4F800C03B4A0325022609275A
:1014B00010300024491CF4452AD11960012907D1B4
:1014C000016841F000710160006800F00070059053
:1014D000106840F0080010601068CDE9005600F078
:1014E0000800CDE9047069462C48CDE9024500F0BA
:1014F0008DF900220521142000F0F8FA142000F0E4
:10150000E7FA00220521152000F0F0FA15203AE054
:10151000DFF88CE0F44538D1D0F800C04CF0806C96
:10152000C0F800C0D0F800C001290CF0806CCDF8E4
:1015300014C0196007D1016841F0007101600068B2
:1015400000F000700590106840F002001060106814
:1015500002AB00F0020005906020CDE9000683E8B0
:10156000B00069460F4800F051F9002205214020E3
:1015700000F0BCFA402000F0ABFA00220521412027
:1015800000F0B4FA412000F0A3FA07B0F0BD00006B
:10159000006400400400002030380240000C02408B
:1015A000006800400004024010B5FFF7E5FB032887
:1015B0000CD000EB800101EBC001054800EB81007D
:1015C000C069002802D0BDE81040004710BD0000EF
:1015D000184A002010B5FFF7CFFB03280CD000EB12
:1015E000800101EBC001054800EB81008069002803
:1015F00002D0BDE81040004710BD0000184A00208E
:1016000010B5FFF7B9FB03280CD000EB800101EB0C
:10161000C001054800EB8100406A002802D0BDE807
:101620001040004710BD0000184A002010B5FFF719
:10163000A3FB03280CD000EB800101EBC00105489F
:1016400000EB8100006A002802D0BDE8104000478E
:1016500010BD0000184A002010B5FFF78DFB0328CD
:101660000CD000EB800101EBC001054800EB8100CC
:10167000806A002802D0BDE81040004710BD00007D
:10168000184A002070B5044690F82000012804D0C4
:10169000606A40F40020606218E0022084F82000B4
:1016A0002068016821F00101016000F0ADF90546F4
:1016B0000EE000BF00F0A8F9401B0A2808D9606AB4
:1016C00040F400306062052084F82000012070BDE5
:1016D00020684068C007EDD1606270BD10B5FFF7AB
:1016E0004BFB03280CD000EB800101EBC001054847
:1016F00000EB8100C068002802D0BDE81040004720
:1017000010BD0000184A002010B5FFF735FB032874
:101710000BD000EB800101EBC001044850F8210020
:10172000002802D0BDE81040004710BD184A002034
:1017300010B5FFF721FB03280CD000EB800101EB73
:10174000C001054800EB81000069002802D0BDE817
:101750001040004710BD0000184A002010B5FFF7E8
:101760000BFB03280CD000EB800101EBC001054806
:1017700000EB81004068002802D0BDE8104000471F
:1017800010BD0000184A002010B5FFF7F5FA032835
:101790000CD000EB800101EBC001054800EB81009B
:1017A0004069002802D0BDE81040004710BD00008D
:1017B000184A002010B5FFF7DFFA03280CD000EB21
:1017C000800101EBC001054800EB81008068002822
:1017D00002D0BDE81040004710BD0000184A0020AC
:1017E00010B5FFF7C9FA03280CD000EB800101EB1C
:1017F000C001054800EB8100C06A002802D0BDE8A6
:101800001040004710BD0000184A00202DE9F84F95
:10181000DFF8BCA10022012503264FF00F090AF1D1
:10182000040BAAF1040E00BF0B6805FA02F4234072
:10183000A34270D10F7907F00307012F01D0022FC7
:1018400016D187684FEA420806FA08FC27EA0C0717
:10185000D1F80CC00CFA08FC4CEA070CC0F808C020
:101860004768A7430C79C4F3001494403C43446098
:101870000C79E443A4070AD0C4684FEA420C06FA84
:101880000CF7BC438F6807FA0CF72743C7600C7945
:1018900004F00304022C12D1D40800EB840CDCF811
:1018A00020405707FF0E09FA07F824EA0804D1F888
:1018B000108008FA07F848EA0408CCF82080046889
:1018C0004FEA420C06FA0CF7BC430F7907F0030706
:1018D00007FA0CF7274307604C6814F4403F70D0B8
:1018E0003C4C276847F480472760246822F00307B0
:1018F00004F480440094384C07EB040CDCF80848EE
:1019000097074FEA177809FA08F7BC43334FB842F4
:1019100002D1002724E054E0314FB84201D1012721
:101920001EE0304FB84201D1022719E02E4FB842D5
:1019300001D1032714E02D4FB84201D104270FE055
:101940002B4FB84201D105270AE02A4FB84201D1F6
:10195000062705E0284FB84201D1072700E00827F5
:1019600007FA08F72743CCF80878DAF8004057461A
:10197000D1F804C09C435FEACC2C00D51C433C60EA
:10198000DBF800405F46D1F804C09C435FEA8C2C32
:1019900000D51C433C60DEF800407746D1F804C017
:1019A0009C435FEA8C3C00D51C433C60084F083FD9
:1019B0003C68D1F804C09C435FEACC3C00D51C4392
:1019C0003C60521C102AFFF42FAFBDE8F88F0000D6
:1019D000083C014044380240003001400000024011
:1019E0000004024000080240000C024000100240C7
:1019F0000014024000180240001C02400AB181613C
:101A000070470904FBE70000014880687047000048
:101A10000800002002488168027811448160704704
:101A2000080000200B4810B5016841F40071016006
:101A3000016841F480610160016841F480710160D6
:101A4000032000F073F80F2000F006F800F024F8EF
:101A5000002010BD003C024070B50D4D04464FF40F
:101A60007A712878B1FBF0F00A490968B1FBF0F00F
:101A700000F01EFB48B9102C07D200222146501E50
:101A800000F034F800206C6070BD012070BD0000D3
:101A900008000020140000200C4882B0016841F4C6
:101AA00080410160006800F4804000900748001FFA
:101AB000016841F0805101600068002200F0805010
:101AC00000900F21901E02B000F010B84438024080
:101AD000002809DB00F01F0201219140400980002D
:101AE00000F1E020C0F8001170470000F0B40E4B88
:101AF0001B680C46C3F30223C3F10705042D00D96C
:101B00000425191D072901D2002300E0DB1E012650
:101B100006FA05F1491E214099409E40761E164066
:101B20003143F0BC00F079BC0CED00E0064900F058
:101B3000070208684FF6FF03184040EA0220034AF4
:101B400010430860704700000CED00E00000FA054B
:101B50002DE9F0470E46050065D0DFF81481D8F86E
:101B60000000F7B200F00700B04207D288F800701A
:101B7000D8F8000000F00700B04254D128683D4C6E
:101B8000810712D5400703D5206840F4E05020605B
:101B90002878000703D5206840F460402060206862
:101BA000A96820F0F000084320602878C0072DD0F5
:101BB000304968680839012812D0022813D0032858
:101BC00011D00968890700292DDA216821F0030165
:101BD00001432160FFF718FF814641F2883A0EE089
:101BE00009688903EFE709688901ECE7FFF70CFF53
:101BF000A0EB0901514502D90320BDE8F087206818
:101C0000696800F00C00B0EB810FEFD1D8F800103C
:101C1000404601F00701B14207D90770006800F0A3
:101C20000700B04201D00120E7E72878400705D53A
:101C30002068E96820F4E050084320602878000715
:101C400006D52068296920F4604040EAC100206080
:101C500000F018F82168084AC1F30311515CC8402C
:101C60000649086006480068FFF7F6FE0020C4E752
:101C7000003C0240083802401049000814000020CF
:101C80000C000020154810B5006810F00C02144834
:101C900013D01449042A0FD0082A0ED10F4C241F48
:101CA0002268236802F03F025B0207D52068C0F378
:101CB0008810A0FB010106E0084610BD2168C1F3B1
:101CC0008811A1FB00010023FEF7DCFA2168C1F3B3
:101CD0000141491C4900B0FBF1F010BD0838024039
:101CE0000024F400001BB7002DE9F84F04006ED06B
:101CF0002078DFF84C93C007A9F104054AD009F118
:101D000004000168C1F38101012908D00068C0F313
:101D1000810002280AD1D9F80000400206D52868BF
:101D2000800337D560680028E1D033E06068B0F503
:101D3000803F10D0B0F5A02F286810D020F480305C
:101D40002860286820F4802028606068A8B1FFF728
:101D50005BFE06460DE0286840F48030F4E740F46E
:101D600080202860F7E700BFFFF74EFE801B642845
:101D700073D828688003F7D50CE0FFF745FE0646C8
:101D800005E000BFFFF740FE801B6428F0D82868FC
:101D90008003F7D42078DFF8AC8280074FF0000A88
:101DA0003ED5A748001D016811F00C0F08D000684F
:101DB000C0F3810002280BD1D9F80000400207D4FB
:101DC0002868800716D5E068012800D112E033E1C9
:101DD000E068B8B10120C8F80000FFF715FE06461C
:101DE00005E000BFFFF710FE801B0228C0D828685E
:101DF0008007F7D52868216920F0F80040EAC10083
:101E000028600DE0C8F800A0FFF7FEFD064604E0DC
:101E1000FFF7FAFD801B02281FD828688007F7D437
:101E20002078000722D5864F87486169703771B1E5
:101E300001210160FFF7E8FD064604E0FFF7E4FD3D
:101E4000801B022809D838688007F7D50EE0C0F853
:101E500000A0FFF7D9FD064605E082E0FFF7D4FDBC
:101E6000801B02287DD838688007F7D42078400787
:101E700068D5DFF8CCB100270BF13C0BDBF8000094
:101E8000C0000BD4DBF8001041F08051CBF80010FB
:101E9000DBF80000012700F0805000906B4E3068A6
:101EA000C00510D4306840F480703060FFF7ACFD9E
:101EB000009005E0FFF7A8FD0099401A022850D8CD
:101EC0003068C005F6D55E4EA0686C3601280FD08C
:101ED0000528306810D020F001003060306820F014
:101EE00004003060A068B8B1FFF78EFD00900FE0ED
:101EF000306840F00100F4E740F004003060F7E79C
:101F0000FFF782FD0099411A41F28830814266D87C
:101F100030688007F4D50EE0FFF776FD009007E00B
:101F2000FFF772FD0099411A41F28830814256D87C
:101F300030688007F4D42FB1DBF8001021F0805115
:101F4000CBF80010A069C8B33D49091D0968C1F369
:101F5000810102294AD00228504607D0C8F8600003
:101F600000E03CE0FFF750FD04463BE04746C8F880
:101F70006000FFF749FD064605E000BFFFF744FD9E
:101F8000801B02282BD828688001F7D4D4E90701E8
:101F90000843A16A2E4A490802EB0141626A41EAFC
:101FA0008211084394F82C1040EA0161C9F800102E
:101FB00001203866FFF728FD044606E03EE000BF3A
:101FC000FFF722FD001B022809D828688001F7D5F9
:101FD00034E000BFFFF718FD001B022802D90320E0
:101FE000BDE8F88F28688001F4D427E00128F7D0F5
:101FF000D9F80000E26900F4800191421CD1226A04
:1020000000F03F01914217D147F6C071626A01406A
:10201000B1EB821F10D1A26A4FF0FF3300F44031C0
:1020200003EB5202B1EB024F06D194F82C1000F0F2
:102030007060B0EB016F01D00120D1E70020CFE745
:102040000438024000004742800E474200700040C2
:102050000000FFFF70B5040003D06079002510B1C7
:1020600005E0012070BD2571204600F00DF802202A
:1020700060712068016841F0040101600120607115
:10208000A560002070BD000008B5006806498842C0
:1020900008D10648016841F040010160006800F085
:1020A0004000009008BD000000080650343802408F
:1020B00010B5401EB0F1807F01D3012010BD4FF05C
:1020C000E02460610F21601700F0A7F90020A061F3
:1020D00007202061002010BDFEE70000104810B569
:1020E0000E4901600321416000214FF4A02281606C
:1020F000C0E903124FF4C002426101760122427628
:102100008176C27601774177FFF733F9002803D053
:10211000BDE81040FEF775BE10BD00000064004031
:10212000E4000020104810B50E4901600321416011
:1021300000214FF4A0228160C0E903124FF4C002D5
:1021400042610176012242768176C276017741773B
:10215000FFF70FF9002803D0BDE81040FEF751BE8D
:1021600010BD0000006800400C01002010B5074AB7
:102170000021074800F020FD0649074A0860BDE835
:1021800010400021054800F017BD0000EC48000891
:10219000492200080000002020490008752300089B
:1021A00070B586B014216846FEF7B6F81A480025C7
:1021B000016841F002010160016801F0020105912E
:1021C000016841F001010160016801F00101059120
:1021D000016841F008010160016801F00801059102
:1021E000016841F08001016000680C4E00F0800041
:1021F0004FF4E0540590002221463046FFF7FEFBE5
:102200000121CDE90041CDE9021569463046FFF7CD
:10221000FDFA06B070BD000030380240001C0240DC
:10222000074910B5054808600846FFF713FF002866
:1022300003D0BDE81040FEF7E4BD10BD0008065015
:1022400034010020FEE7FEE710B500F0B3FCBDE866
:10225000104000F0F6BC000010B5094C607808B1E1
:10226000002010BD03224FF480710020FEF728FCEF
:1022700010B14FF0FF3010BD01206070F0E700009A
:10228000A800002010B50B4888B04FF0FF3440780C
:1022900038B100236A464FF480711846FEF756FBAA
:1022A00010B1204608B010BD0DF10D0001F050F93D
:1022B0000020F7E7A800002010B5FFF7ABFB02F005
:1022C0001BF9012803D0BDE8104001F0C3BC10BDCC
:1022D00030B593B030216846FEF71EF814210CA8E3
:1022E000FEF71AF81D480025016841F08051016091
:1022F000006800F0805011901948016841F4804155
:1023000001600068022400F48040119001200090D8
:10231000000401908001CDE9064006200890A82025
:10232000CDE9090407200B906846FFF7DDFC08B1F2
:1023300072B6FEE70CA90F2081E831004FF4A050DF
:102340000F904FF48050109005210CA8FFF700FC6F
:10235000002801D072B6FEE713B030BD403802400D
:10236000007000400248016841F47001016070474C
:1023700088ED00E010B500F0BDFA0A4A00210A48D5
:1023800000F01AFC094C00220A212060022000F013
:1023900033FB606000F0E0FA00F00CFCBDE8104098
:1023A00000F04FBC44490008B1230008B84B00209E
:1023B00000F08AFAFEF7D1F89FED131B53EC112BB6
:1023C000FEF75CF8FEF7D6F80546052000F051FA56
:1023D00000F073FA0446FEF7EBFAFFF73DFF0C48F6
:1023E00001210022017041708270C1702C44FFF7FE
:1023F00049FF084800F074F80548FEF7CFFC204676
:1024000000F044FAF2E7000000000000000059402C
:10241000DC000020A04A0020FEE70907090E002882
:1024200004DB00F1E02080F80014704700F00F009A
:1024300000F1E02080F8141D704700B52DED048BED
:10244000B0EE409AF0EE609A83B051EC190BFEF7B3
:102450009EF941EC180B18EE100A18EE901A8DED4B
:10246000008B002818BF0120084320F00040C0F175
:102470007F6000F1E040C00F14D019EE101A19EE81
:10248000900A8DED009B002918BF0121084320F020
:102490000040C0F17F6000F1E040C00F04BF0120A8
:1024A00000F018F8B0EE480A03B0F0EE680ABDEC90
:1024B000048B00BD02E008C8121F08C1002AFAD12F
:1024C00070477047002001E001C1121F002AFBD1B4
:1024D000704700000149086070470000E0000020DC
:1024E0002DE9F04706462DED088B00F089F99FEDA8
:1024F000940A9449944C88B3944802794088012AFC
:1025000002D000280BD814E000EE100AF8EE400AC2
:1025100094ED010AF4EEC00AF1EE10FA09DD00EEC6
:10252000900AB8EE601AC0EE010AC4ED050A20EE6A
:10253000200A84ED020A94ED040A10EE100A884283
:102540000DDADFED830A30EEC00ADFED820A20EEFD
:10255000200ABCEEC00A10EE100A01E00EE00020D6
:102560002070C0B200F0EEFF2078D4ED020A00EE39
:10257000100AB8EE400A30EEC00A0DE0D4ED040AAD
:1025800010EE900A884207DA9FED731A60EE810A16
:10259000C4ED060A20EE200A002084ED020A94ED24
:1025A000030A9FED6E2A6E4FDFED6E8A9FED6E9AE5
:1025B000DFED6E9AC0EB001106EB8101D1ED060A4A
:1025C00006EB8001D1F8F01060EEA81A91ED001A28
:1025D00007EB800161EE811A61EE092A42EE811A51
:1025E00020EE821A41EE201A71EEA90AC1ED000A0E
:1025F000F5EEC00AF1EE10FA01D330EE800A401C6D
:10260000C0B20428D6D384ED030AD4ED020AB4EE96
:10261000E00AF1EE10FA6BDD80EE801ADFF84081FF
:10262000002508F1100884ED051A9FED51AB00BF9D
:1026300007EB8500D4ED050A90ED000A08EB850054
:1026400020EE200A80ED000AB5EEC00AF1EE10FA85
:102650004AD306EB8500D0F8F000D0ED000A20EE5A
:10266000891A20EEA88A11EE200A70EE290A28EEB7
:10267000080A9FED411A00EEC10AB5EEC00AF1EE5C
:1026800010FA31D3C5EB051006EB800910EE100AE5
:10269000D9ED060AF5EEC00AF1EE10FA2CDDFDF7D1
:1026A00082FF41EC100BFFF7C8FEF0EE60BAF1EECE
:1026B000480AB0EE40BA10EE900AFDF774FF53ECF2
:1026C0001B2BFDF734FE53EC1A2BFDF7D7FEFDF75D
:1026D0007DFF00EE100A294910EE100A884201DD44
:1026E0009FED270A89ED060A6D1CEDB2042D9FD3DC
:1026F000BDEC088BBDE8F087FDF755FF41EC100BF2
:10270000FFF79BFEB0EE40BAB1EE480AF0EE60BAB9
:1027100010EE100AFDF747FF53EC1B2BFDF7A8FE48
:1027200053EC1A2BFDF7AAFEFDF750FF00EE100A3E
:10273000144910EE100A8842D4D99FED130AD1E74C
:102740000000000000004842C0000020B800002047
:1027500000004842CDCC4C3E0AD7A33CFC110434C7
:10276000804A00204F020636C3031C348D978240F6
:10277000000000803F82903EFC11043500007A4644
:1027800000007A4600007AC600007AC62DE9F041C2
:10279000040006D0184E306884420AD10020BDE8FB
:1027A000F081502080F31188BFF34F8FBFF36F8FFC
:1027B000FEE700F041FF6569776BB66B00F05CFFE8
:1027C000BD4201D0B54201D10220E8E70B48854265
:1027D00008D1A06A0028F7D194F858000128F3D056
:1027E0000320DCE705481438854202D00DB10120F2
:1027F000D5E70420D3E700001800002034060020AD
:1028000010B5FFF701F90F499FED0F1A88604A686C
:10281000801A01F11002D279424300EE102AB0F57D
:102820007A7FF8EE400A91ED030AB8EE400A00EE16
:10283000810ABCEEC00A81ED030A01D9002010BD57
:10284000012010BDA80000206F12833AFFF7EAF8BC
:10285000FFF73EFDFFF7A4FCFFF740FCFFF762FC2B
:10286000FFF7DEFC00F034F8FFF780FC00F058F8CA
:10287000FEE710B5EFF3058111B16FF0050403E039
:10288000002408B100F0B0FF204610BD38B5054661
:10289000EFF3058010B16FF005040CE0002401F0A7
:1028A00039FE291A0090002903DD684600F0C2FFB6
:1028B00001E06FF00304204638BDEFF3058008B156
:1028C00001F02EBE01F026BE4FF47A707047000072
:1028D000EFF3058010B16FF0050070470448016800
:1028E00011B14FF0FF3070470121016000207047A7
:1028F0006800002010B5EFF3058010B16FF00500FF
:1029000010BD01F0F9FD20B1022804D04FF0FF30D6
:1029100010BD012010BD01F0E9F8002010BD00003D
:1029200010B5EFF3058010B16FF0050010BD084839
:102930000168012902D04FF0FF3010BD054A002187
:1029400082F8141D0221016001F08CF8002010BDF6
:10295000680000200BE000E070B5EFF3058010B1D7
:102960006FF0050413E001F0C7FD4FF0FF3510B123
:1029700002280BD108E0012401F0F2FE012806D064
:1029800001F0BAFD10B102E0002400E02C46204620
:1029900070BD0000F8B51D466FF003026FF002062F
:1029A0004FF00004EFF30583A3B1F0B1E9B1E5B94D
:1029B000002200926A4601F0DDFB012817D1009841
:1029C000B0B10C494FF080500860BFF34F8FBFF398
:1029D0006F8F0DE048B141B12A4601F02FFB01286D
:1029E00006D025B16FF0010402E0144600E0344641
:1029F0002046F8BD04ED00E0F8B514464FF00005A0
:102A0000EFF3058212BB08B301B3A4B1D4E90232DB
:102A100063B1502A1AD32269C2B1676900FB01F67B
:102A2000B74213D3009501F064F907E072B9226947
:102A300062B9626952B9002201F03AF9050005D085
:102A40000CB1216800E0002100F098FE2846F8BD96
:102A5000F8B51D466FF003026FF002064FF0000458
:102A6000EFF30583ABB100B3F9B1F5B9002213461A
:102A700000926A4601F064FA012818D10098B8B1B2
:102A80000C494FF080500860BFF34F8FBFF36F8F3A
:102A90000EE050B149B100232A4601F0A1F9012806
:102AA00006D025B16FF0010402E0144600E0344680
:102AB0002046F8BD04ED00E02DE9F0410D46014649
:102AC00021F0010001F001014FF00004EFF3058255
:102AD0000AB1A41F16E048B100296FF001066FF09B
:102AE0000207294608D001F04FFC07E06FF003040D
:102AF00008E035B1344605E001F08AFB0128F8D141
:102B000000E03C462046BDE8F08170B505464FF038
:102B10000004EFF3058050BB0DB1686800E00020B1
:102B2000C10701D0012600E0002600071FD46DB1C7
:102B3000D5E9021021B1502819D31EB1042002E0BA
:102B400020B114E0012001F0A6F805E00EB1042048
:102B500000E0012001F094F8040008D00DB12968CC
:102B600000E0002100F00AFE0EB144F0010420460E
:102B700070BD70B5014621F0010001F001014FF078
:102B80000004EFF305820AB1A41F11E028B16FF031
:102B9000020529B101F033FA07E06FF0030407E002
:102BA00000231A46194601F01BF9012800D02C46D3
:102BB000204670BD01F09ABC2DE9FF414FEA0103A8
:102BC0004FF00005EFF30581039549BB40B3802723
:102BD000182100244AB3166806B1344696691EB11E
:102BE0003146761E382E02D21679F60703D0002021
:102BF00004B0BDE8F081566906B1B708D2F808C044
:102C0000BCF1000F0DD0D5685C2D18D312693AB114
:102C100036B18DE806103A46214601F03CFC03909F
:102C20000DE0D6685EB912694AB903AACDE900126F
:102C3000BAB2214601F002FC012800D003950398A6
:102C4000D6E770B50546EFF3058010B16FF00504C7
:102C50000FE04DB12846FFF799FD042807D0002466
:102C6000284600F02DFE04E06FF0030401E06FF051
:102C70000204204670BD00002DE9F041134C0F46C0
:102C80000546E6682068001D00F07AFC681C07D144
:102C900037B12168BDE8F0410D48091D00F0C0BC06
:102CA00020683544B5424560216805D2A06BBDE877
:102CB000F041091D00F09CBC606B091D00F098FC00
:102CC000A06A854200D2A562BDE8F081180000200C
:102CD000340600202DE9F041054600F0ADFC2D4CF6
:102CE000A068401CA06020682B4F10B1606930B311
:102CF0002BE02560A068012827D1002606EB86007E
:102D000007EB800000F066FC761C382EF6D32348D3
:102D100000F060FC2148143000F05CFC1F482830B3
:102D200000F058FC1D483C3000F054FC1B4850306B
:102D300000F050FC194860631430A06305E020687F
:102D4000E96AC06A884200D82560606A401C6062F7
:102D50006864E86A2169884200D9206100EB80003C
:102D600007EB8000291D00F05BFC00F085FC60692A
:102D700000280CD02068E96AC06A884207D2084956
:102D80004FF080500860BFF34F8FBFF36F8FBDE8E7
:102D9000F08100001800002084010020E4050020DC
:102DA00004ED00E038B500F047FC104C2068C8B9CD
:102DB0000F4800F00FFC0E48143000F00BFC0C48DC
:102DC000E060143020610A4B0020F03B009003F1DA
:102DD000500210210A2000F08CFF206010B105A1E4
:102DE00000F0CCFCBDE8384000F046BC54000020A8
:102DF00038070020546D72510000000030B4026C9E
:102E00000B46002A0BD0C1681144C1608468A142FE
:102E100001D30168C16030BC1846FDF764BA30BC0C
:102E200070472DE9F041856B174604460026026C79
:102E300082B1C7B1E068FDF756FAE168206C091A63
:102E4000E1602268914202D2A168081AE060022F74
:102E500016D017E02068A8B9A06801F0CDFB06469F
:102E60000020A0600EE06068FDF73DFA216C60680C
:102E700008446060A168884204D32068606001E073
:102E800005B16D1E6D1CA5633046BDE8F08110B51F
:102E9000044690F8590058B101280CD002280FD0F0
:102EA000502080F31188BFF34F8FBFF36F8FFEE781
:102EB000206B00F0F5FB2046BDE8104000F0F0BBB1
:102EC00010BD000010484FF47051420706D0C01DDD
:102ED0000D4920F00700411AC1F570510B4A00233B
:102EE0000144C2E900030839183A21F007011160D2
:102EF0004B600B600B1AC0E9001393604FF0004069
:102F00005360506170470000180E002084000020BC
:102F1000144E154CA6F29C474FF08058DFF84C90A9
:102F200012E000BF00F088FBF068C568281D00F0C3
:102F300027FBA068401EA0606068401E606000F033
:102F40009BFB2846FFF7A3FF60680028EAD138689A
:102F50000128F9D9C9F80080BFF34F8FBFF36F8FF5
:102F6000F2E70000200600201800002004ED00E039
:102F7000002807D00021816001600B460A46C1602D
:102F800000F02EBF7047000070B51D46049C51B183
:102F9000C4F80020C4E90F010121204600F0DCFE46
:102FA00084F84C5070BD2460F4E700002DE9F05F18
:102FB0008846DDE90B941546834691009A460A9EA1
:102FC000A522206BFDF7A1F96FF00301206B01EB47
:102FD0008501084420F00707780707D0502080F3C8
:102FE0001188BFF34F8FBFF36F8FFEE70025B8F155
:102FF000000F0FD05FF00000221818F8001082F8C0
:10300000341018F8001011B1401C1028F4D384F8C3
:10301000435001E084F83450382E00D33726E6625E
:10302000C4E91365201D00F0E0FA04F1180000F077
:10303000DCFA2461C6F138006462A061656584F839
:10304000585052465946384600F066FA2060B9F1A9
:10305000000F01D0C9F80040BDE8F09F30B511491C
:1030600000E011460A688242FBD34B685C18844238
:1030700003D1406818444860084643681C189442CD
:1030800009D1084C183C2468A24209D052681A445D
:1030900042600A6812680260814200D0086030BD58
:1030A0000460F9E78400002070B5002441600B4DF6
:1030B0000061914206D8D11A8269914206D2011D5F
:1030C000286907E09A4203D2994201D3012403E020
:1030D000011DE86800F08CFA204670BD5400002005
:1030E00010B5044600F0A8FAA06B28B15FF0000408
:1030F00000F0C2FA204610BD0124F9E730B589B0CE
:103100003C4D6EE00498002806DADDE90601059AD8
:1031100090470498002864DB069C606910B1201D6C
:1031200000F02EFA03A800F0D7F8024604980A2807
:1031300057D2DFE800F00505052D334A05052D338C
:1031400094F8280040F0010084F828000599A0694F
:10315000059B01442046FFF7A7FF68B3216A20467C
:10316000884794F8280040073BD500200090059838
:10317000A169002342181946204601F083FBD8B903
:10318000502080F31188BFF34F8FBFF36F8FFEE79E
:1031900014F8280F20F00100207022E094F8280095
:1031A00040F0010084F828000598A06128B181183A
:1031B00013462046FFF778FF13E0502080F3118874
:1031C000BFF34F8FBFF36F8FFEE794F8280081079E
:1031D00003D4204600F064FA03E020F0010084F8F4
:1031E0002800002204A9286800F028FF002889D1BF
:1031F00009B030BD540000202DE9FC410F460546C2
:1032000000F074FC01A800F067F80446019818B1BA
:1032100001F0A6FABDE8FC81254EAFB13069006827
:10322000D0B30027291B3A46306800F0BBFA01F002
:1032300097FA0028EED11F494FF080500860BFF385
:103240004F8FBFF36F8FE5E7A542EBD801F088FA07
:10325000F0682746C068C468201D00F091F994F812
:103260002800410719D5A0692B4641193A46204646
:10327000FFF71AFFA8B100200346014600902A4636
:10328000204601F0FFFA60B9502080F31188BFF3A7
:103290004F8FBFF36F8FFEE707E020F0010084F847
:1032A0002800216A20468847B4E70127BAE70000D2
:1032B0005400002004ED00E00648416B096829B184
:1032C000416BC968C9684968816270474FF0FF3136
:1032D000FAE700001800002070B5054601F01AF961
:1032E000064E0446B068844203D200F009F801207B
:1032F00000E0002028602046B46070BD540000202B
:10330000F8B5194D20E0C068C4680668201D00F0BB
:1033100037F9216A2046884794F82800400713D5DA
:10332000A0693044B04206D924616060211DE8687C
:1033300000F05EF908E000200346014600903246A6
:10334000204601F09FFA38B1E86801680029DAD117
:103350002969C5E90310F8BD502080F31188BFF337
:103360004F8FBFF36F8FFEE754000020084840687E
:10337000401C4FF0500080F3118804D0BFF34F8FF2
:10338000BFF36F8FFEE7BFF34F8FBFF36F8FFEE783
:103390008C000020074CE068016841B1C068002142
:1033A000D0F80000FFF728FFFFF7A8FEF3E70121A0
:1033B0000020F7E7540000202DE9F041044600F01A
:1033C0003BF994F9455004F1240609E0606A48B1DC
:1033D000304601F08DF908B100F0C2FA6D1E6DB2F1
:1033E000002DF3DC4FF0FF3684F8456000F044F91F
:1033F00000F022F994F9445004F1100709E0206923
:1034000048B1384601F074F908B100F0A9FA6D1E10
:103410006DB2002DF3DC84F84460BDE8F04100F0AB
:103420002BB900002DE9F0410546002700F05EFBB6
:10343000324E306808B9FFF745FD706905424ED13C
:10344000C5B3083568070ED005F00700C0F10800C5
:103450000544680707D0502080F31188BFF34F8FD1
:10346000BFF36F8FFEE72DB37068854237D82348CE
:10347000183001460C6801E020460C466168A942FC
:1034800002D221680029F7D131688C4227D0076821
:103490002168016060680837411B10290FD9601945
:1034A000420708D0502080F31188BFF34F8FBFF33D
:1034B0006F8FFEE713E041606560FFF7CFFD616845
:1034C0007068401A7060B268904200D2B060706953
:1034D00001430020C4E90001F068401CF06001F0E5
:1034E0003FF9780707D0502080F31188BFF34F8F42
:1034F000BFF36F8FFEE73846BDE8F0816C00002017
:103500000449086818B10868026D521C0265086811
:10351000704700001800002010B5031F4FF08074A2
:103520001C601B1F21F001011960191F044B0B6067
:1035300014390A60091F6FF0020244380A6010BD96
:103540006D3300080149087070470000A800002092
:1035500010B50446FEF758FA084948600748217834
:103560001030017161784171A1780170E1784900F2
:103570004180217981716179C17110BDA80000205D
:10358000D0E9013201699A60D0E901235A604A68A2
:10359000824201D182684A60002202610868401EAE
:1035A0000860086870470000034B036003F15C008B
:1035B000086080201060704760070020044B0360A3
:1035C00003F15C0008604FF48070106070470000E9
:1035D000BC09002000F108014FF0FF32C0E90112E0
:1035E000C1600161002101607047002101617047E5
:1035F00030B50B685A1C02D000F1080202E00269E3
:1036000004E02246546825689D42FAD953684B600D
:1036100099608A60516008610168491C016030BD91
:1036200042684A6093688B60936859609160086152
:103630000168491C01607047502080F31188BFF376
:103640004F8FBFF36F8F0A494868401C48600128BC
:103650000CD10848006810F0FF0F07D0502080F30D
:103660001188BFF34F8FBFF36F8FFEE770470000E5
:103670008C00002004ED00E00849486828B1401E95
:10368000486001D180F311887047502080F3118881
:10369000BFF34F8FBFF36F8FFEE700008C00002059
:1036A00070B500282AD0164DA0F108046068696939
:1036B000084207D1502080F31188BFF34F8FBFF32A
:1036C0006F8FFEE722683AB1502080F31188BFF374
:1036D0004F8FBFF36F8FFEE78843606000F006FAFC
:1036E00060686968084468602046FFF7B7FC28698D
:1036F000401C2861BDE8704001F032B870BD000088
:103700006C0000204FF0E02000210161816105493B
:103710004FF47A720968B1FBF2F1491E4161072149
:10372000016170471400002010B5FCF795FD1149A8
:1037300010280ED300F1E02090F8F0030A789042B0
:1037400007D2502080F31188BFF34F8FBFF36F8FE4
:10375000FEE709480068896800F4E060884207D9FC
:10376000502080F31188BFF34F8FBFF36F8FFEE7B8
:1037700010BD00008C0000200CED00E010B5084BDF
:10378000002200BF53F832401CB1521C082AF9D362
:1037900010BD43F8321003EBC201486010BD0000B9
:1037A0004401002070B515460E460446FFF744FF5D
:1037B00094F944100020491C01D184F8440094F984
:1037C0004510491C01D184F84500FFF755FFA06B57
:1037D00028B92A46314604F1240000F0DFF82046DB
:1037E000BDE87040FFF7E8BD10B5020014D00F48E7
:1037F000006B38B1502080F31188BFF34F8FBFF3B7
:103800006F8FFEE700F072F900211046FFF734FADF
:1038100000F0A6FF002807D105494FF0805008604E
:10382000BFF34F8FBFF36F8F10BD00001800002053
:1038300004ED00E070B50D4604000BD095B11E4AB2
:10384000106BB8B1502080F31188BFF34F8FBFF3D6
:103850006F8FFEE7502080F31188BFF34F8FBFF3C7
:103860006F8FFEE7502080F31188BFF34F8FBFF3B7
:103870006F8FFEE700F03AF9D26823685919934236
:1038800004D98B420AD9914202D807E08B42FAD977
:10389000881A21600021FFF7EFF900E0216000F0B5
:1038A0005FFF002807D105494FF080500860BFF343
:1038B0004F8FBFF36F8F70BD1800002004ED00E044
:1038C00070B50546FFF7B8FE1E4C05B92568281DE2
:1038D000FFF756FEA86A18B105F11800FFF750FE71
:1038E000606A401C60622068854207D1291D164825
:1038F000FFF796FE6068401C606007E0A068401E0D
:10390000A0602846FFF7C3FAFFF7D6FCFFF7B4FE26
:103910006069002814D02068854211D1206B38B12D
:10392000502080F31188BFF34F8FBFF36F8FFEE7F6
:1039300006494FF080500860BFF34F8FBFF36F8F81
:1039400070BD0000180000202006002004ED00E0FB
:1039500002490A6A0260C968416070471800002085
:1039600001490120C86170471800002010B50C46BD
:1039700050B1094909681831FFF73AFE2046BDE801
:1039800010400121FFF778B9502080F31188BFF370
:103990004F8FBFF36F8FFEE71800002070B51446FD
:1039A0000D4668B10A4909681831FFF739FE0CB1B4
:1039B0004FF0FF3521462846BDE87040FFF75CB95F
:1039C000502080F31188BFF34F8FBFF36F8FFEE756
:1039D0001800002070B504003ED0226DA2B1E06C4A
:1039E000884200D30146E06A884235D0012A33D1AB
:1039F0001A4D2A6894420FD1502080F31188BFF3EA
:103A00004F8FBFF36F8FFEE7502080F31188BFF315
:103A10004F8FBFF36F8FFEE7E162A269002A02DBDE
:103A2000C1F13801A1610E4E00EB8000616906EB27
:103A30008000814210D1201DFFF7A2FDE06A2969B4
:103A4000884200D9286100EB800006EB8000211D30
:103A5000BDE87040FFF7E4BD70BD00001800002015
:103A60008401002030B587B00024039405AA04A97E
:103A700003A80494FFF798FDDDE903010094CDE964
:103A80000110002315A11748059A00F004FD164DFA
:103A90000028E8621FD000F0C5FE012809D0401CB4
:103AA00019D1502080F31188BFF34F8FBFF36F8F70
:103AB000FEE7502080F31188BFF34F8FBFF36F8F65
:103AC0004FF0FF30A86201206861EC6007B0BDE8EC
:103AD000304000F045B807B030BD000049444C45C7
:103AE00000000000112F0008180000200248016BA0
:103AF000491C01637047000018000020164810B5EB
:103B0000016B11B10121C16110BD0021C1610169C9
:103B1000124A01E0B9B1491E01EB810352F823308A
:103B2000002BF7D001EB810302EB830202F10804C2
:103B300053685B685360A34201D15B685360DA68E5
:103B40000260016110BD502080F31188BFF34F8FD8
:103B5000BFF36F8FFEE700001800002084010020F3
:103B60001CB537480168374A914207D1502080F38D
:103B70001188BFF34F8FBFF36F8FFEE700683149A5
:103B8000491E884207D1502080F31188BFF34F8F20
:103B9000BFF36F8FFEE72C4908780190FF20087073
:103BA00008788DF800009DF800009DF8002000F0D6
:103BB000F000904207D0502080F31188BFF34F8F60
:103BC000BFF36F8FFEE79DF80000204C00F050001F
:103BD00020700720A06005E09DF8002052008DF8BD
:103BE0000020401E9DF800201206F5D4A060032896
:103BF00007D0502080F31188BFF34F8FBFF36F8F32
:103C0000FEE74FF44070A060019808700C48203027
:103C1000016841F470010160016841F07041016088
:103C2000FFF770FD00206060FCF7DEFA08480168CD
:103C300041F040410160FCF7C3FA00201CBD0000C8
:103C400000ED00E071C20F4100E400E08C000020B4
:103C500034EF00E010B5502080F31188BFF34F8F90
:103C6000BFF36F8F00F064FC18B104494FF080502F
:103C70000860002080F3118810BD000004ED00E012
:103C800010B502460021012000F012F80446FFF7AB
:103C90006FF9204610BD38B50B4600220090114642
:103CA000012000F026F80446FFF762F9204638BDEF
:103CB000F8B517460E46050013D005FB06F0503048
:103CC000FFF7B0FB04000AD0002084F8460004F19E
:103CD00050023B46314628460094FFF755F92046EE
:103CE000F8BD502080F31188BFF34F8FBFF36F8F63
:103CF000FEE738B5049D18B153B1CAB181B120E0D7
:103D0000502080F31188BFF34F8FBFF36F8FFEE712
:103D1000502080F31188BFF34F8FBFF36F8FFEE702
:103D2000502080F31188BFF34F8FBFF36F8FFEE7F2
:103D300039B1502080F31188BFF34F8FBFF36F8FDD
:103D4000FEE750241C46012384F846302B4600949D
:103D5000FFF71AF9204638BD70B50D46040025D08E
:103D6000FFF76AFCD4E90F20216802FB0011A16073
:103D70000021A163216861600A46D4E90F01401E59
:103D800000FB0121E16021464FF0FF3001F8440FB4
:103D9000487004F110008DB1FFF71CFC04F1240001
:103DA000FFF718FCFFF768FC012070BD502080F37E
:103DB0001188BFF34F8FBFF36F8FFEE72169002992
:103DC000F0D000F095FC0028ECD004494FF0805072
:103DD0000860BFF34F8FBFF36F8FE3E704ED00E0A0
:103DE0002DE9FF4782B01D468A464FF000080400C7
:103DF00003D0BAF1000F08D011E0502080F31188F1
:103E0000BFF34F8FBFF36F8FFEE7206C38B15020A8
:103E100080F31188BFF34F8FBFF36F8FFEE7022D42
:103E20000AD1E06B012807D0502080F31188BFF33E
:103E30004F8FBFF36F8FFEE700F05EFB3F4F4FF0F9
:103E400000094FF0805648B9049838B1502080F3EB
:103E50001188BFF34F8FBFF36F8FFEE7FFF7ECFBC7
:103E6000A06BE16B884207D3022D05D00498D0B136
:103E7000B8F1000F1AD01EE02A4651462046FEF740
:103E8000D0FF616A19B104F1240000F031FC20B1C7
:103E90003E60BFF34F8FBFF36F8FFFF7EDFB012045
:103EA00006B0BDE8F087FFF7E7FB22E06846FFF7C2
:103EB0004FFD4FF00108FFF7DFFBFFF717FEFFF79D
:103EC000BBFB94F94400401C01D184F8449094F960
:103ED0004500401C01D184F84590FFF7CDFB04A9B3
:103EE000684600F071FA30B12046FFF765FA00F03D
:103EF00037FC0020D4E7FFF79FFBA06BE16B884203
:103F000013D1FFF7B9FB04F110000499FFF72EFD60
:103F10002046FFF751FA00F023FC00289ED13E60B6
:103F2000BFF34F8FBFF36F8F98E7FFF7A5FB2046D6
:103F3000FFF742FA00F014FC90E7000004ED00E007
:103F40002DE9F0471F4690468946040003D0B9F199
:103F5000000F08D011E0502080F31188BFF34F8F7D
:103F6000BFF36F8FFEE7206C38B1502080F31188CB
:103F7000BFF34F8FBFF36F8FFEE7022F0AD1E06BC5
:103F8000012807D0502080F31188BFF34F8FBFF373
:103F90006F8FFEE7FFF7C8FB5020EFF3118680F329
:103FA0001188BFF34F8FBFF36F8FA06BE16B884217
:103FB00006D3022F04D0002086F31188BDE8F087D5
:103FC00094F94550A06B3A4649462046FEF729FF32
:103FD000681C04D06D1C84F845500120ECE7606A31
:103FE0000028FAD004F1240000F082FB0028F4D06D
:103FF000B8F1000FF1D00121C8F80010EDE710B5BD
:10400000040009D000F072FAA168884214D1E06877
:10401000401EE06008D00DE0502080F31188BFF30F
:104020004F8FBFF36F8FFEE700231A4619462046D5
:10403000FFF7D6FE012010BD002010BD2DE9F74787
:10404000002683B08A46040003D0BAF1000F08D0DE
:1040500011E0502080F31188BFF34F8FBFF36F8FB3
:10406000FEE7206C38B1502080F31188BFF34F8FEA
:10407000BFF36F8FFEE700F03FFADFF8F4804FF0F8
:1040800000094FF0805748B9059838B1502080F3A7
:104090001188BFF34F8FBFF36F8FFEE7FFF7CCFAA6
:1040A000A56BC5B151462046FEF7A8FE6D1EA5635F
:1040B000206950B104F1100000F01AFB28B1C8F8D3
:1040C0000070BFF34F8FBFF36F8FFFF7D5FA01205A
:1040D00006B0BDE8F087059808B11EB106E0FFF70D
:1040E000CBFA27E06846FFF733FC0126FFF7C4FA56
:1040F000FFF7FCFCFFF7A0FA94F94400401C01D143
:1041000084F8449094F94500401C01D184F845900E
:10411000FFF7B2FA05A9684600F056F900282046D4
:104120000AD0FFF749F900F01BFB2046FEF7D8FF45
:104130000028B3D00020CBE7FEF7D2FF90B104F106
:1041400024000599FFF712FC2046FFF735F900F02F
:1041500007FB0028A2D1C8F80070BFF34F8FBFF350
:104160006F8F9BE72046FFF727F900F0F9FA95E7F4
:1041700004ED00E02DE9F04790468946040003D0A5
:10418000B9F1000F08D011E0502080F31188BFF37F
:104190004F8FBFF36F8FFEE7206C38B1502080F354
:1041A0001188BFF34F8FBFF36F8FFEE7FFF7BCFAA5
:1041B0005020EFF3118680F31188BFF34F8FBFF3C8
:1041C0006F8FA76BF7B194F9445049462046FEF72C
:1041D00015FE7F1EA763681C04D06D1C84F8445034
:1041E000012010E020690028FAD004F1100000F04E
:1041F0007FFA0028F4D0B8F1000FF1D00121C8F8FF
:104200000010EDE7002086F31188BDE8F08700007C
:104210002DE9F343002683B00400354609D0206C15
:1042200078B1502080F31188BFF34F8FBFF36F8FA9
:10423000FEE7502080F31188BFF34F8FBFF36F8FDD
:10424000FEE700F059F9DFF83C814FF000094FF02C
:10425000805748B9049838B1502080F31188BFF3D3
:104260004F8FBFF36F8FFEE7FFF7E6F9A06BC8B182
:10427000401EA063206810B9FFF742F9A0602069D2
:1042800050B104F1100000F033FA28B1C8F8007002
:10429000BFF34F8FBFF36F8FFFF7EEF9012005B02B
:1042A000BDE8F083049808B166B10FE03DB150203D
:1042B00080F31188BFF34F8FBFF36F8FFEE7FFF7D7
:1042C000DBF95DE06846FFF743FB0126FFF7D4F911
:1042D000FFF70CFCFFF7B0F994F94400401C01D142
:1042E00084F8449094F94500401C01D184F845902D
:1042F000FFF7C2F904A9684600F066F800282046D6
:1043000012D0FFF759F800F02BFA2046FEF7E8FE2E
:104310000028A9D09DB3FFF78FF9606A50B3206BD6
:104320000068C0F1380126E0FEF7DAFEE0B120684F
:1043300038B9FFF781F9A06800F09EF90546FFF74C
:104340009BF904F124000499FFF710FB2046FFF7C6
:1043500033F800F005FA002886D1C8F80070BFF3E2
:104360004F8FBFF36F8F7FE72046FFF725F800F0F0
:10437000F7F979E70021A068FFF72CFB9FE7FFE73B
:1043800000208CE704ED00E070B50D46040009D074
:1043900000F0ACF8A16888420CD1E068401CE060F5
:1043A000012070BD502080F31188BFF34F8FBFF301
:1043B0006F8FFEE729462046FFF72AFF0028F0D03E
:1043C000E168491CE16070BD2DE9F0410C46050033
:1043D00011D0C4B1FFF730F9174BDA686E68206866
:1043E000911B471C17D02F681B6A9F4219D0964219
:1043F00017D8012410E0502080F31188BFF34F8FAD
:10440000BFF36F8FFEE7502080F31188BFF34F8F0B
:10441000BFF36F8FFEE70024FFF72EF92046BDE8BB
:10442000F081884205D9401A20602846FFF790FAAB
:10443000F1E700202060DCE7180000202DE9FF5F95
:104440008346DDE90E87994616468A469000FEF7B8
:10445000E9FF05001CD05C20FEF7E4FF040014D047
:104460000020256384F85900CDE90240CDE900879A
:104470004B46324651465846FEF798FD2046FEF719
:1044800029FC012004B0BDE8F09F2846FFF708F999
:104490004FF0FF30F6E7F0B585B0DDE90B640A9D1B
:1044A000A6B1DCB15C2700972663022684F8596028
:1044B000002604AFCDE90246CDE90057FEF776FDB0
:1044C0002046FEF707FC049805B0F0BD502080F3AD
:1044D0001188BFF34F8FBFF36F8FFEE7502080F33B
:1044E0001188BFF34F8FBFF36F8FFEE7014800685D
:1044F00070470000180000200548416919B1006BA1
:1045000018B100207047012070470220704700005A
:10451000180000200148C068704700001800002003
:1045200010B5FFF701F90148C06810BD1800002060
:104530002DE9F0412E4C0027206B28B1A069401CCA
:10454000A0613846BDE8F081E668761CE66013D1CC
:10455000606B006838B1502080F31188BFF34F8F33
:10456000BFF36F8FFEE7606BA16B6163A063206A8E
:10457000401C2062FEF7A0FEA06ADFF87880864229
:1045800009D3606B0068A0B1606BC068C5686868DB
:10459000864211D2A0622068C06A00EB800158F800
:1045A0002100012800D90127E0690028C9D001278E
:1045B000C7E74FF0FF30EDE7281DFEF7E1FFA86ADF
:1045C00018B105F11800FEF7DBFFE86A216988429F
:1045D00000D9206100EB800108EB8100291DFFF765
:1045E0001FF8E86A2168C96A8842CAD30127C8E768
:1045F000180000208401002070B504004FF0000175
:1046000033D01B4D2868844207D0502080F3118896
:10461000BFF34F8FBFF36F8FFEE7206D38B1401EA1
:104620002065E36CE26A9A421FD040B11DE0502041
:1046300080F31188BFF34F8FBFF36F8FFEE7201D0C
:10464000FEF79EFFE06CE062C0F13800A061E06A16
:104650002969884200D92861064900EB800001EBF6
:104660008000211DFEF7DCFF0121084670BD00001F
:10467000180000208401002070B504004FF00000F5
:104680002BD0194DE16A2A68D26A914226D2A069DC
:10469000002804DB2868C06AC0F13800A061134E0E
:1046A00001EB8101606906EB8101884211D1201D77
:1046B000FEF766FF2868C06AE0622969884200D96F
:1046C000286100EB800006EB8000211DFEF7A8FFAB
:1046D00002E02868C06AE062012070BDE16C2A68CF
:1046E000D26A9142F8D370BD1800002084010020E6
:1046F00070B5C068C46854B104F118000646FEF7EE
:104700003FFF144D286B50B13146134815E050203F
:1047100080F31188BFF34F8FBFF36F8FFEE7201D2B
:10472000FEF72EFFE06A2969884200D928610B490B
:1047300000EB800001EB8000211DFEF771FFE06AB5
:104740002968C96A884202D90120E86170BD002049
:1047500070BD0000180000200C060020840100201D
:104760002DE9F0472C4D00242746286B38B1FEF781
:1047700063FF286B401E2863286B40B146E0502041
:1047800080F31188BFF34F8FBFF36F8FFEE7A968E7
:10479000224E0120D1B3A6F5916980463068E0B180
:1047A000F068C46804F11800FEF7EAFE201DFEF769
:1047B000E7FEE06A2969884200D9286100EB8001A0
:1047C00009EB8100211DFEF72BFFE06A2968C96A09
:1047D0008842E3D3C5F81C80E0E70CB1FEF76CFD1E
:1047E000AC694CB14FEA0806FFF7A2FE00B1EE61DA
:1047F000641EF9D10020A861E86938B10849012791
:1048000038070860BFF34F8FBFF36F8FFEF734FF99
:104810003846BDE8F0870000180000200C06002094
:1048200004ED00E010B586B0FEF7BCFA114C20682C
:10483000B8B100200390049005AA04A903A8FEF7CC
:10484000BDFEDDE9032102208DE8070000230AA157
:104850000B48059AFFF71FFE606010B106B00120FB
:1048600010BD502080F31188BFF34F8FBFF36F8FBF
:10487000FEE7000054000020546D72205376630060
:10488000953300082DE9FF411E46134602000A9D9C
:104890004FF0000016D0144C2768002F0FD0CDE940
:1048A00000130292062917DAFFF726FE02284FF0BE
:1048B00000030FD0002269462068FFF791FA04B088
:1048C000BDE8F081502080F31188BFF34F8FBFF314
:1048D0006F8FFEE72A46EEE70023324669463846E8
:1048E000FFF72EFBEBE700005400002068490008AA
:1048F00000000000000000000000000000000000B8
:10490000000200001800000000000000000000008D
:10491000000000000000000001020304060708096F
:1049200074490008000000000000000000000000C2
:104930000000000000040000300000000000000043
:104940000000000080490008000000000000000096
:10495000000000000000000000040000180000003B
:10496000000000000000000064656661756C74540E
:1049700061736B005461736B5F496E697400000072
:104980006361705F6374726C00000000AC490008E2
:1049900000000020E4000000B4240008904A000851
:1049A000E4000020F44E0000C424000800000000D1
:1049B00000000000010000001000000000000000E6
:1049C0000024F400000000000000000000000000CF
:1049D00000000000000000000000000000000000D7
:1049E00000000000000000000000000000000000C7
:1049F00000000000000000000000000000000000B7
:104A000000000000000000000000000000000000A6
:104A10000000000000000000000000000000000096
:104A20000000000000000000000000000000000086
:104A3000000000000000000000000000AAAAAAAACE
:104A40000000000000000000000000000000000066
:104A50000000000000000000000000000000000056
:104A60000000000000000000000000000000000046
:104A70000000000000000000000000000000000036
:104A80000000000000000000000000000000000026
:040000050800018965
:00000001FF
